:100000000BC018951895189518951895189518956A
:1000100018951895189518958FED8DBFC0ECE4EBE9
:100020004E2EDD275D2EEEE7F0E0A0E6B0E0A895CD
:1000300084B7082E877F84BF88E1992781BD91BD51
:1000400088278D933197E9F766248DEF8ABB8FED72
:1000500087BB80E08BBB80E088BBD99A83E886B9F8
:1000600080E087B980E080936800A3E6F2D280E068
:100070008093670080E080936200ACE6E8D28091D4
:1000800074008F7780937400D198A4E79C9196FFB9
:1000900004C0C99B0EC09F7B9C93C9990AC084E68B
:1000A0009F93992780D19F91C99903C090649C9395
:1000B00016D1AEE6CCD2379A81E080936B000091E6
:1000C0006B000A3010F009F020C0EF93FF93E5E1D8
:1000D000F0E060D1FF91EF9107B1007E086007B9B1
:1000E00071D1ACE68D939C93AEE60D911C91ACE67C
:1000F0004D915C91040F151FAEE60D931C93ABE67A
:100100008C918F5F8C9308F4DACF3798EEE6F0E0AD
:10011000D190E080FF240027B6D1A0E7E5D1EEED35
:10012000F6E08CD2E0E7F0E08AD154D2EDE0A0E72F
:10013000A0D2E2EEF6E082D2E0E7F0E080D14AD24F
:10014000EDE0A0E796D2E6EEF6E078D2E0E7F0E068
:1001500076D1EAD1EDE03FD1A0E6DC92ACE60D919C
:100160001C910C3B52E0150708F004C0A0E68C91EE
:100170008D5F8C93009160004AE0A1D2A1E60C93C0
:1001800000916100003010F009F001C001C02CD0D6
:1001900084E690E008D100916700043009F022C0A5
:1001A000A4E78C9187FB0EF00DC0EAE0F0E0A3E637
:1001B00094E07BE76CD25FD0809174008F7780935E
:1001C000740053CFEAE0F0E0A4E194E071D2A3E63A
:1001D0000D911D912D913C9147D209F002C072C042
:1001E00001C02EC051CF3ECFD89A84E690E0DBD03C
:1001F000D89884E690E0D7D0A7E68C918F5F8C9357
:10020000A3E60D911D912D913C914AE050E060E0F4
:1002100070E07AD0A3E60D931D932D933D93A3E652
:100220000D911D912D913C91A1E64C91552766278A
:10023000772715D2A3E60D931D932D933D93089533
:1002400084E690E0B0D0A8E68C918F5F8C9389E033
:10025000809369008FE580936A0018D00091680050
:10026000033009F007C0ECE3F0E048D080E0809371
:10027000680001D0FACE84E690E095D082E08093C9
:10028000690088EC80936A0001D0089581E0809332
:100290006B004091690000916B00041710F009F0A9
:1002A00010C0D89AAAE68C9199277DD0D898AAE652
:1002B0008C91992778D0ABE68C918F5F8C9308F462
:1002C000E8CF0895D8DF8CE291E06DD0DA9AE2E0D1
:1002D000F0E014D0DA98E1E0F0E010D0C6CED89A81
:1002E00084E690E060D0D89884E690E05CD080917D
:1002F0007400806880937400BEDF089588EE93E0F8
:1003000052D03197D9F7089522D006D000FC01D001
:10031000089528D030D00895842F952FA62FB72F79
:100320004427552766277727F1E2889409C020F4EF
:10033000480F591F6A1F7B1F7695679557954795FC
:100340003795279517950795FA9589F7089500240D
:10035000E89477FF02C006D0689400F809D010F83E
:100360000124089512D04F5F5F4F6F4F7F4F089564
:10037000E89437FF089500951095209530950F5F0C
:100380001F4F2F4F3F4F68940895409550956095AB
:10039000709508953197F1F70895689462F808957B
:1003A000E89462F80895EF93FF93EE27E82BE92B8A
:1003B00031F0EAEFF0E03197F1F70197D1F7FF91D3
:1003C000EF910895369A3699FECF369A3699FECF38
:1003D00084B195B1089533D0992711278F2D880FB7
:1003E00080E8F82A802F881F08F41FEF41F08F570C
:1003F000082F07FD04C0003240F08FEF01C08827AE
:10040000982FD82EE82EF82E09C08FE1801B082FD8
:10041000F694E794D79497950A95D1F7112351F064
:100420009095D094E094F09481E0980F8827D81E9E
:10043000E81EF81E0F2DFE2CED2CD92E0895D1901C
:10044000E190F19001910895219131914191519163
:100450000895102F90E8FF0C001F0927990FF794BB
:100460001078652F90E8440F551F5927990F47952D
:10047000607800380895FF0C90E89027110F979549
:10048000F794092F0895102FBD2CDE2CEF2CF02EA1
:1004900011234AF4B094D094E094F0949FEFB91AE9
:1004A000D90AE90AF90A0EE1FF2039F4FE2CED2CF5
:1004B000DB2CBB240850C2F76BC032F00A95BB0C92
:1004C000DD1CEE1CFF1CF9CF01D0D5CFB7FE08957F
:1004D00090E8B91611F4D0FE08959FEFD91AE90AF1
:1004E000F90A09F403950895DD92ED92FD920C93BB
:1004F0000895502F2D2D3E2D4F2D612F08952DEC59
:100500003CEC4CEC5DE366270FC099DFF2DFDD24A5
:10051000EE2490E8F92E0FE307C096DF05C02227EE
:10052000332740E251E46627552351F1002381F13E
:1005300090DF71F11627005850580894050B18F4F5
:1005400007FD03C025C007FD23C0469537952795B5
:10055000F694E794D79422D0FF202AF0DD0CEE1C0D
:10056000FF1C015073F09D2D969548F0DD203AF464
:10057000EE202AF491E0D90E9927E91EF91E7BCFCF
:1005800007C09FE7092FF92A9FEFD92EE92E08957A
:10059000DD24EE24FF240027112708959F9299243B
:1005A000AA24BB2488E1D216E306F40628F0D21A66
:1005B000E30AF40A089401C08894991CAA1CBB1C85
:1005C000DD0CEE1CFF1C8A9571F7D92CEA2CFB2C54
:1005D0009F9008953EDFE1F25038D1F2162700587F
:1005E00050580894051F12F418F4CBCF08F0D0CF60
:1005F0000AD0FF202AF0BB0CDD1CEE1CFF1C3BCFF9
:100600000F5FFBF138CF9F929924AA24BB2499272E
:1006100088E1990CAA1CBB1CDD1CEE1CFF1C30F4ED
:10062000920EA31EB41ED91EE91EF91E8A9589F7E3
:100630009F900895C895319600200895FBDF202DE6
:10064000F9DF302DF7DF402DF5DF502D089582E0E2
:1006500001C084E099279D938A95E9F70895040FD6
:10066000151F261F371F089504171507260737077C
:10067000089594E081918D939A95E1F70895E19919
:10068000FECFEEBB3196089591E001C092E07B373A
:1006900051F47FB7F894F3DF8D918DBBE29AE19A24
:1006A0009A95C9F77FBF7727089591E001C092E03E
:1006B000E6DFE09A8DB38D939A95D1F70895FF9375
:1006C000881BF9E0001FFA9511F4FF910895881F27
:1006D000841B18F4840F8894F5CF0894F3CF0AD7BD
:0A06E000A33B00009A420000804096
:00000001FF
